:020000040800F2
:10500000401C0020D55000089D90000877860008BD
:105010000000000000000000000000000000000090
:10502000000000000000000000000000BD9F00081C
:1050300000000000000000008D9A0008F9A00008A0
:10504000E7500008E7500008E7500008E750000864
:10505000E7500008255C0008E7500008E75000080A
:1050600000000000E7500008315B0008E75000082E
:10507000E7500008AD8B000800000000E750000872
:1050800000000000E75000080000000000000000E1
:10509000E750000800000000E7500008E750000853
:1050A000E7500008E7500008E7500008ADAB0008E3
:1050B000E7500008E7500008000000000000000072
:1050C0000348854600F07EFC00480047ADBC000860
:1050D000401C00200448804704480047FEE7FEE7E4
:1050E000FEE7FEE7FEE7FEE7B9A10008C1500008B1
:1050F00030B50B46014600202022012409E00D4670
:10510000D5409D4205D31D469540491B25469540F7
:1051100040191546521E002DF1DC30BD70B500243B
:105120002546002801DA01244042002901DA012540
:105130004942FFF7DDFFAC4200D04042002C00D0D6
:10514000494270BDF0B51FB40646002082B0054646
:105150004024019100901BE0019922460F46304601
:1051600000F06CFB049A059B801A994110D31046FD
:105170001946224600F052FB361A8F41019722460B
:1051800001200021009F00F049FB38184D4100909C
:105190002046641E0028DFDC019B00982946324629
:1051A00007B0F0BD03460B439B0703D009E008C9D5
:1051B000121F08C0042AFAD203E00B780370401CC7
:1051C000491C521EF9D27047D2B201E00270401C55
:1051D000491EFBD270470022F6E710B513460A4677
:1051E00004461946FFF7F0FF204610BD30B50446CF
:1051F0000020034600E05B1C934203D2E05CCD5CE0
:10520000401BF8D030BDF8B502464A40D40F4200EA
:105210004B0052085B089A4202D2024608461146E9
:105220004A0023D0C30D4A00DDB2120EAD1A202D64
:1052300035DA49020126490AF6058A19002C00D000
:10524000524220214F1B1146B9402A411018C20D6D
:105250009A4221D0002C17D0012D08DCDA05801AE3
:10526000D20F8019D207DBB200F014FBF8BDDA05CB
:10527000801A012340001B06C01880185A4280186B
:10528000CA0F1043490007E04908C2071143DA0575
:10529000801A80194008801800F0F4FAF8BD610007
:1052A0000122511A001BF7E70122D2075140AAE759
:1052B0000122D2075040A6E770B502464A40D50FFA
:1052C00040004A00ED0740085208002814D0002A88
:1052D00012D0C40DD30D41020120C0055202490A6B
:1052E000520AE41A091812187D34914201D3641C41
:1052F00000E04900002C01DA002070BD002391423B
:1053000001D3891A0343400849000028F7D1002936
:105310000AD0914202D10121C90705E0914201D290
:10532000012101E00121C943E005C018401900F046
:10533000A9FA70BDF0B507460846584087B0C00FBF
:10534000049048000E46590040084908BC1A88419C
:1053500005D2384631461E4617460B4602465800CF
:10536000400810434CD0300D039040055900400DCB
:10537000490D0590401A0290402872DA1803012165
:10538000000B09050843019004980092002805D0FD
:1053900001995242002088410092019002984021D8
:1053A0000A1A0199009800F039FA05460C466B4636
:1053B00007CB00F054FAC0197141039A0E0D002377
:1053C000D71756401A467A40164344D0049A002A0A
:1053D0002DD0029A012A039A15DC1205C01A9141B8
:1053E00001263605001C7141D20F059ED20700939D
:1053F000019202962A46234600F092FA07B0F0BDC9
:1054000038463146FAE71605224A0F46B218C01A46
:10541000B74101210905001C4F4100187F41114689
:1054200018187941E20F10436D19644113E0E20747
:105430006D0815436408C2071443039A0126120538
:10544000C01A91413605001C7141CE074008304317
:105450004908C01851412A46234600F054FACDE7C6
:10546000FFE7049801224000C117121A00238B4164
:1054700004983146C417381AA141EEE730B401242C
:10548000E407634030BC55E730B40124E4076140D1
:1054900030BC4FE70000E0FFF0B51FB488B00B99B7
:1054A0000998002448400999C00F4900490809910A
:1054B000C0070B990090490049080B910999089879
:1054C000A64608431CD00B990A98084318D009989F
:1054D00001244000420D4800410D099824050003B5
:1054E000000B204309900B980003000B20430B9006
:1054F00050181C494018002201901446104605E03F
:10550000002001460DB0F0BD032801DA034600E09B
:1055100003239C46C11A0AAE0AE05F0008ADED5BAA
:105520004F00F75B7D430027AA187C41491C5B1E96
:105530006145F2DD410004AB5A522104120C0A43CA
:10554000240C401C0828DFDB01980290009970466B
:1055500001910090059B049A0799069800F0E0F9E4
:10556000D0E700000DFCFFFFF0B50C465C4085B0B5
:10557000E40FE40703944C000026640859009446A5
:10558000490802460296224321D062460A431ED0B1
:105590006200570D4A000E032303550D01240246F5
:1055A0002C492405781B1B0B360B4018234326433C
:1055B000614600901C46501AB44103D30098401C29
:1055C000009002E0921800985B41002803DA002066
:1055D000014605B0F0BD00200121090507468646B9
:1055E00011E064461D46141BB54106D36546521BA7
:1055F000B341744607430C43A646CD07400849080B
:10560000284392185B4105460D43EAD110461843E2
:1056100013D06046194650407140084306D060469A
:10562000101AB34106D20122002306E00022012312
:10563000DB0702E00122D2435310009874460105B3
:10564000381C6141029C039D0019694100F05BF91F
:10565000BFE70000FD030000C217C10F504010B5A6
:105660004018CA079623002100F014F910BD10B5A8
:1056700000229623114600F00DF910BD0EB5C21799
:10568000C10F5040CA0740180021054B02930192F8
:1056900000910A460B4600F043F903B000BD00003C
:1056A000330400000EB505490291002100910A461D
:1056B0000B46019100F034F903B000BD3304000043
:1056C000410040020122400AD205090E80187F29BC
:1056D00001DA00207047962903DC9622511AC8404F
:1056E000704796398840704770B5CD0F4A0009035E
:1056F0000123090B1B0519430B4BED070024520D29
:105700009A4201DA002070BD074B34339A4203DC21
:105710009A1A00F093F802E00449511888402C438B
:10572000F1D0404270BD0000FF030000CDFBFFFF41
:105730004A0009030123090B1B051943094B10B546
:10574000520D9A4201DA002010BD064B34339A42C2
:1057500003DC9A1A00F072F810BD03495118884012
:1057600010BD0000FF030000CDFBFFFFC20FD207FA
:10577000400040080BD0C10D0723DB01C9184002CF
:105780000905400A1143C208400711437047002031
:105790000146704710B5002904DB0124E4074042AC
:1057A0008C412146002B04DB1C460123DB075242BF
:1057B000A341994200D1904210BD0000CB0FDB07FE
:1057C000490010B5490802460A4307D00A0D0724CC
:1057D0000903E401090B121B002A01DC002010BDA3
:1057E000C900440F0C43C100E018D205801800F036
:1057F00049F810BD0122D207002800DB101A002949
:1058000000DB511A814270470122D207002800DBD9
:10581000101A002900DB511A8842704710B5202A5F
:1058200004DB0146203A9140002010BD9140202326
:105830009C1A0346E3401943904010BD10B5202A3E
:1058400004DB0846203AD040002110BD0B46D3406F
:10585000D0402024A21A91400843194610BD10B52B
:10586000202A06DBCB170846203A1041C1170B430C
:1058700006E00B461341D0402024A21A9140084371
:10588000194610BD002904DA401C490001D1400826
:105890004000704770B40024050C05D110240004AA
:1058A00002D1002921D01124050E01D100020834B3
:1058B000050F01D10001241D850F01D18000A41C1A
:1058C000002801DB4000641C002908D020252E1B85
:1058D0000D46F540A14000D00121294308430106AF
:1058E0001B1B000ADB1D02D5002070BC7047DB05C6
:1058F000181880180029F8DA401C4900F5D170BC4E
:1059000040084000704710B5002B08DA0024401C06
:10591000614192185B411A4301D14008400010BD1B
:10592000F0B51FB482B005460C0003D0084605F060
:105930006BFA02E005F068FA20300246009021463A
:105940002846FFF76BFF049B059A04460F46184351
:105950001143084314D0184610431BD0009840212F
:105960000A1A18460599FFF769FF05460E46009A80
:1059700005990498FFF752FF084305D0012004E081
:105980002046394607B0F0BD0020C11705430E433D
:105990002C43374300990E986305401A7905E40AB1
:1059A00000220C43FD0A0A3002D500200146E9E737
:1059B0000105101969410C9C0D9D00196941FFF703
:1059C000A2FFDFE7064C0125064E05E0E36807CCA1
:1059D0002B430C3C98471034B442F7D3FFF774FBC9
:1059E00070C0000890C0000870B58C180578401C85
:1059F0006B075B0F01D10378401C2A1106D1027896
:105A0000401C03E006780E70401C491C5B1EF9D157
:105A10002B0705D40023521E0DD40B70491CFAE746
:105A20000378401CCB1A921C03E01D780D70491CB2
:105A30005B1C521EF9D5A142D8D3002070BD0000D6
:105A400038B50446074908480068FFF751FB604332
:105A5000009002E00098401E009000980028F9D1C4
:105A600038BD000040420F008801002070B5044698
:105A70000025206880688007800F012807D12068F2
:105A80000068C007C00F002801D0012000E00020FE
:105A9000002839D1206880681C490840002801D1BD
:105AA000012000E00020002809D1606D102108438A
:105AB0006065A06D01210843A065012070BD2068CC
:105AC000806801210843216888600120FFF7B8FF42
:105AD00001F014FA05460EE001F010FA401B0A2806
:105AE00009D9606D102108436065A06D012108434C
:105AF000A0650120E2E720680068C007C00F01210F
:105B0000484048400028E7D00020D7E71700008031
:105B100010B502460B460020002103E0545C241817
:105B2000A0B2491C9942F9D3C443A0B210BD0000F1
:105B300010B5034800F0DCFE024800F0D9FE10BDAD
:105B4000DC1700209417002030B51C25446C2C4035
:105B50000125A540046C6560046863608468102CAE
:105B600004D10468A2600468E16003E00468A160F5
:105B70000468E26030BD000001201749487202202D
:105B80001649487203201649487204201549487284
:105B9000114815490A7842714978817110481249B3
:105BA0000A784271497881710C480F490A7842702D
:105BB000497881700B480C490A78427049788170A5
:105BC0000A4809490A7842704978817006490A787A
:105BD0004271497881717047BC1100201A1200206F
:105BE000DE110020D01100204401002030120020DE
:105BF00010B504F0B7F9202004F06CFA012005F08C
:105C00001FFD002004F066FA044805F087FB0448F5
:105C100005F0B8FE002005F0F5FE10BD6100002083
:105C20008380000010B501210520000701F052F922
:105C3000002802D000200C49086002210B4801F026
:105C400049F9002809D108490860094800880A2153
:105C500048430849088004F0BBFF012001F034F8F4
:105C6000022001F031F810BD800100200004005036
:105C700060010020740100207047000000210A4AE2
:105C800051610A494968012252021143074A516091
:105C90001146496808221143044A51600021C20993
:105CA000D20111607047000024180020002002403B
:105CB0007FB504460D460020039000F0BDFF002094
:105CC00000900194E809029003A9684600F036FFAD
:105CD000002804D000F078FF002004B070BD00F070
:105CE00073FF0120F9E710B50346002002E01C5CB9
:105CF0000C54401C9042FAD310BD000000203949DA
:105D00008969FF2201321140914208D1364949691F
:105D100002221143344A5161FF21013108433149C4
:105D20008969012252021140914208D12E494969E4
:105D3000012211432C4A516101214902084329499A
:105D40008969012292021140914208D1264949698C
:105D500008221143244A5161012189020843214943
:105D600089690122D2021140914208D11E49496934
:105D7000042211431C4A51610121C90208431949F7
:105D80008969012252031140914208D1164949699B
:105D900010221143144A516101214903084311495A
:105DA0008969012252041140914207D10E49496983
:105DB000202211430C4A5161202108430949896975
:105DC000012212041140914208D107494969402239
:105DD0001143054A516101210904084301498861C1
:105DE00070470000002002402418002070B50446CF
:105DF00001F084F805460BE0601C002808D0002C58
:105E000004D001F07BF8401BA04201D9032070BDF3
:105E10001F488069C007C00F0028EDD11C48806969
:105E200002210840022801D1194988611848806977
:105E3000FF2101310840884223D01548806949007C
:105E4000084088421DD012488069490008408842B5
:105E500017D00F48806949000840884211D00C488B
:105E600080698900084088420BD00948806909018F
:105E70000840884205D00648806949100840884299
:105E800003D1FFF73BFF0120C1E70020BFE700007F
:105E900000200240F0B585B006460F4614460025A6
:105EA000029601970020009000F0C6FE13E00198D2
:105EB000006803900220039A029900F095FE00907A
:105EC0000098002800D008E00298001D0290019878
:105ED000001D01902D1DA542E9D300BF00F074FE06
:105EE000A54202D2002005B0F0BD0120FBE7000072
:105EF0000246002108E04800064B185A904201D1A2
:105F000008467047481CC1B2034800788142F2DB62
:105F100000BFF6E72A1400202801002070B50446CF
:105F20000D462946204600F0DEFF70BDFEB50C4848
:105F300001F0F2F980B202900298FFF7B3FB044639
:105F4000084A094BFFF7A8FA0022084B019100907C
:105F5000FFF70AFB0646FFF7EBFB80B2FEBD000031
:105F60008C160020F853E3A59B843E4000408F40F0
:105F700010B5454845490A784270497881704449CE
:105F80000A7842714978817105203F49487296200C
:105F900005F0E6FC4B20C00005F0FEFC00223A496B
:105FA0000C2005F0FBFD00210C2005F00BFE02206B
:105FB00005F030FD00BF00210F2005F029FC354918
:105FC0000860354908400028F5D032480068401C78
:105FD000002801D103F0A0F82E48006801218903B0
:105FE000084000283FD08122D20100210F2005F077
:105FF0008EFD0021102005F00BFC4406640E2146A6
:106000000022264805F054FC2448407A05283AD15D
:1060100002221F492148401DFFF7E8F8002832D12D
:106020001E48807A1E49087004221C49491C1D48DC
:10603000FFF7B8F81B48006800F042F81A490880DA
:1060400017480078420015490B311848FFF7AAF8A5
:1060500015480088164909884843164908800220D7
:10606000154908700FE0104908880988491E0E4B31
:10607000198012490988FFF751F80D4800884143FB
:1060800088B20C49088010BD3012002002010020A7
:10609000440100207000002000D02724801200203E
:1060A0002801002030010020FC0000202A140020DC
:1060B00056010020520100206000002058010020FD
:1060C00070B50646174801F027F9C5B22846E9170A
:1060D000C90E091849114901691ACCB209E03046C4
:1060E000E040C007C00F002801D1204670BD601CF1
:1060F000C4B20D4800888442F1DB012409E0304637
:10610000E040C007C00F002801D12046EEE7601C28
:10611000C4B2054800888442F1DB03480078401E81
:10612000C0B2E3E78C1600205801002010B50B48E0
:1061300000F074FB0A21094800F0FAFA074800F061
:10614000A1F9012149020840884204D1034800F026
:106150009CF980B210BD00BFFCE7000030160020A3
:10616000F0B587B000220121424800F0C0FEFFF7E1
:10617000DDFF0546FFF77BFA04463F49FFF79CF831
:106180003E490860012211463A4800F0B0FE3B4803
:106190000068FFF7EBFA04460022394BFFF7FAFAE2
:1061A0005ED838480078002821D000203549087092
:1061B000FFF7BCFF0546FFF75AFA04462E49FFF7E2
:1061C0007BF82E49086008460068FFF7CFFA0446BE
:1061D00000222B4BFFF752F900222B4B0591049024
:1061E000FFF75AF90646FFF7E9FA284908602348FD
:1061F0000068FFF7BBFA06460022214BFFF73EF985
:106200000446234A234BFFF747F9039102901F48A6
:106210000068FFF7ABFA04461D4A52421E4BFFF7D7
:106220003BF901910090039B029AFFF783F80591D7
:106230000490FFF7C3FA154908601849134800682D
:10624000FFF7E2FA02D215481049086000210F4812
:106250000068FFF7CFFA06D200200C49086002E080
:1062600000200A49086009480068FFF729FAC0B20F
:1062700007B0F0BD0004005000401B44280000207F
:1062800000000C403000002000E064402C000020A2
:106290003333333333B33040CCCCEC3F0000C8420F
:1062A000F8B5044600250026002700BF5020005DF9
:1062B000012801D10220F8BD01215020015500BF65
:1062C000206880688007800F012806D12068006858
:1062D0000840002801D0012000E00020002841D122
:1062E000606DFF2101318843022108436065206809
:1062F000C0688707BF0F2068C068800880002168D9
:10630000C860206880680121C90708432168886047
:1063100000F0F4FD064611E000F0F0FD801B0A28B5
:106320000CD9606D0221884310210843606500BFCD
:1063300000215020015500BF0120BCE72068806883
:10634000C00FC0070121C9078842E5D02068C06896
:1063500038432168C860606D0221884301210843E9
:10636000606504E0606D202108436065012500BF81
:1063700000215020015500BF28469CE770B5044617
:106380000D4600BF5020005D012801D1022070BDE4
:1063900001215020015500BF206880680421084079
:1063A000800800280AD0606D20210843606500BF86
:1063B00000215020015500BF0120E8E72D49686801
:1063C000884229D02068806A29684903490B08431C
:1063D0002168886228684003400B27490840012152
:1063E0008904884208D12548806849010843234927
:1063F00088600A20FFF724FB28684003400B2049EF
:1064000008400121490488422CD11C488068490178
:1064100008431A49886025E02068806A2968490392
:10642000490B88432168886228684003400B124961
:10643000084001218904884205D11048806849013B
:1064400088430E49886028684003400B0C49084087
:1064500001214904884205D10848806849018843E0
:106460000649886000BF00215020015500BF002070
:106470008DE70000011000000000044800270140E3
:10648000000002440146486D704701460868006CF0
:106490007047000010B50446002C01D1012010BD4A
:1064A000606D002806D1A0650021502001552046CE
:1064B00000F00EF9606D10210840102806D0206809
:1064C000806804210840800800280AD0606D1021EF
:1064D0000843606500BF00215020015500BF012026
:1064E000DDE7606DFF2101318843022108436065CB
:1064F000206880688007800F012807D12068006825
:10650000C007C00F002801D0012000E000200028B3
:106510003AD100BF032189076068884207D0494209
:106520006068884203D04900606888420CD12068C6
:10653000006980008008216808612068006961683E
:1065400008432168086112E0206800698000800823
:10655000216808615C4880680F21890488435A4992
:10656000886008468068616808435749886000BFB2
:106570002068C068182188432168C8602068C06806
:10658000A16808432168C8604F4880680121490616
:1065900088434D49886008468068A18E49060843B3
:1065A000494988602068806801210907084000285F
:1065B00004D1206880680843216888602068C0682A
:1065C000424908402168C8602169E068022901D178
:1065D000042100E0002108432021095D490308430C
:1065E0002C21095D49000843216B0843A1698903F7
:1065F0000843E169C90308432168C9680843216861
:10660000C860FF21C231606A884207D0A16A606A0F
:1066100008432168C96808432168C8602120005DDB
:10662000012813D12020005D002807D12068C06810
:106630000121090408432168C86007E0606D20213A
:1066400008436065A06D01210843A065E06B012847
:1066500017D120680069FF218900884321680861FB
:10666000216C606C0843A16C0843216809690843E8
:1066700021680861206800690121084321680861D8
:106680000BE020680069C007C00F002805D0206813
:106690000069400840002168086120684069C0081E
:1066A000C0002168486120684069A16B08432168E7
:1066B00048610020A065606D0221884301210843E4
:1066C00060650020EBE60000002701401902FEFF94
:1066D00010B586B00446142101A8FEF77CFD1249CE
:1066E000206888421ED11148406B491508430F4964
:1066F000486300BF0846C06A012108430B49C862CD
:106700000846C06AC007C00F009000BF00BF02204B
:106710000190032002900020039001A905200007AA
:1067200000F0E2FA06B010BD002401400010024063
:10673000F8B504460D46002600276069082801D1F7
:10674000082711E02068C068C007C00F00280AD0E1
:10675000606D20210843606500BF00215020015575
:1067600000BF0120F8BD0C2700F0C8FB064614E06E
:10677000681C002811D0002D04D000F0BFFB801B46
:10678000A8420AD9606D04210843606500BF00215A
:106790005020015500BF0320E4E72068006838401E
:1067A0000028E5D0606D012149020843606520683A
:1067B000C068032189020840002826D12020005DFE
:1067C000002822D1206800680821084008281CD130
:1067D0002068806804210840800800280DD12068C6
:1067E00040680C21884321684860606DFF210131B9
:1067F000884301210843606507E0606D202108435C
:106800006065A06D01210843A065A069002802D140
:106810000C20216808600020A4E7000070B5044641
:1068200000252068806804210840800800282BD1BA
:1068300000BF5020005D012801D1022070BD012160
:106840005020015500BFE069012803D02046FFF722
:106850000DF90546002D18D1606D0D490840FF2146
:106860000131084360650020A06500BF0021502071
:10687000015500BF1C202168086020688068042141
:1068800008432168886000E002252846D6E700001A
:10689000FEF1FFFF70B5044600252520005D0228AB
:1068A00003D00420E063012520E0206800680E2169
:1068B000884321680860206800684008400021681B
:1068C00008601C21606C084001218140206C4160FF
:1068D00001212520015500BF00212420015500BFC2
:1068E000A06B002802D02046A16B8847284670BDC7
:1068F00070B50446206C0568206806681C20616C31
:10690000014004208840284000281DD00420304049
:10691000002819D02068006820210840002805D1EF
:106920002068006804218843216808601C21606C8D
:10693000084004218140206C4160206B00285AD01F
:106940002046216B884756E01C20616C01400220E4
:1069500088402840002825D002203040002821D03F
:106960002068006820210840002808D120680068BD
:106970000A218843216808600121252001551C2136
:10698000606C084002218140206C416000BF002102
:106990002420015500BFE06A00282CD02046E16A7F
:1069A000884728E01C20616C01400820884028406E
:1069B000002820D00820304000281CD02068006823
:1069C0000E218843216808601C21606C0840012169
:1069D0008140206C41600120E063012125200155A8
:1069E00000BF00212420015500BF606B002802D0A9
:1069F0002046616B884770BD70B50446002C01D1FC
:106A0000012070BD244A2168881A1421FEF770FB0A
:106A10008000606420480838206402212520015548
:106A2000206805681D480540E168A06808432169A1
:106A3000084361690843A1690843E1690843216A81
:106A4000084305432068056001218903A068884246
:106A500017D011487830806A1C22616C11400F22D7
:106A60008A4090430C49783188621C22616C114045
:106A70006068884008497831896A08430649783156
:106A800088620020E0630121252001550021242097
:106A900001550020B5E70000080002400F80FFFF0D
:106AA000F8B504460D4616461F460020009000BF6C
:106AB0002420005D012801D10220F8BD01212420FD
:106AC000015500BF2520005D01282DD10221252080
:106AD00001550020E06320680068400840002168FC
:106AE00008603B46324629462046FFF72DF8206BCA
:106AF000002806D0206800680E210843216808603D
:106B00000BE0206800680421884321680860206841
:106B100000680A2108432168086020680068012194
:106B200008432168086006E000BF002124200155C9
:106B300000BF022000900098BFE70000F8B50446AF
:106B40000E460127002500BF1C48007C012801D10A
:106B50000220F8BD01201949087400BF1848FFF74A
:106B600045F90746002F22D1401E3060656817E0C6
:106B70002846FFF783F81248FFF738F9074611480F
:106B80004068082188430F49486008464068491515
:106B900088430C494860002F01D0356006E08035FD
:106BA000A068C00161684018A842E1D800BF00BFDA
:106BB00000200249087400BF3846CAE724180020A4
:106BC00050C30000002002400648406802210843EC
:106BD000044948600846406801210843014948606B
:106BE0000020704700200240F8B507460C461546C5
:106BF000012600BF0E48007C012801D10220F8BD0B
:106C000001200B49087400BF0A48FFF7EFF8064659
:106C1000002E06D10649486125600648FFF7E6F8D0
:106C2000064600BF00200249087400BF3046E6E770
:106C30002418002050C300001D484068C007C00F42
:106C4000002816D000BFEFF31080014600BF72B6D7
:106C50001848174AD0601848D06000BF81F31088E8
:106C600000BF10464068C007C00F002801D00120B7
:106C700070470F48406802221040022815D100BF1B
:106C8000EFF31080014672B60C48094A10610C48B7
:106C90001061084680F3108800BF10464068022249
:106CA0001040022801D10120E2E70020E0E70000C7
:106CB00000200240EFCDAB8905040302BFAE9D8CDE
:106CC000161514137047000010B5044605484069B6
:106CD0002040002804D0034844612046FFF7F2FF1B
:106CE00010BD00000004014070B5034600220024DE
:106CF0000020DAE0012696400D6835402C46002C35
:106D000077D04D68022D02D04D68122D15D1D508CF
:106D1000AE001D462035A8595507EE0E0F25B5408B
:106D20000646AE4330465607F60E0D69B540284379
:106D3000D508AD001E46203670514D68012D08D093
:106D40004D68022D05D04D68112D02D04D68122DD1
:106D500018D1986856000325B5400646AE43304624
:106D60005600CD68B5402843986058680125954085
:106D70000646AE43304610264D6835402D099540F5
:106D800028435860186856000325B5400646AE43B0
:106D900030460D79AD07AD0F5600B5402843186059
:106DA000D86856000325B5400646AE433046560027
:106DB0008D68B5402843D860012636074D683540B8
:106DC000B54271D13C4D6D6B012635433A4E75632A
:106DD0003A4D9608B600A85995072E0F0F25B540D5
:106DE0000646AE43304605252D07AB4202D10025AD
:106DF00015E059E0324DAB4201D101250FE0314D94
:106E0000AB4201D102250AE02F4DAB4201D103254F
:106E100005E02E4DAB4201D1052500E00625960781
:106E2000360FB5402843254D9608B600A851284D89
:106E300028680546A5432846012636044D68354096
:106E4000B54202D1054625432846214D2860686891
:106E50000546A5432846012676044D683540B542CF
:106E600002D1054625432846194D6860A8680546A5
:106E7000A5432846012636054D683540B54202D166
:106E8000054625432846124DA860E8680546A543F7
:106E90002846012676054D683540B54202D10546A3
:106EA000254328460A4DE860521C0D68D540002D48
:106EB00000D01FE770BD0000001002400800014034
:106EC0000004005000080050000C0050001C00504E
:106ED00000040140024613690B40002B01D0012041
:106EE00000E00020704742694A4042617047002A32
:106EF00001D0816100E081627047000001480068B4
:106F0000704700008401002002480068401C0149CD
:106F1000086070478401002010B50024084800680C
:106F20004021084306490860002000F00BF80028C3
:106F300001D0012401E000F025FA204610BD000038
:106F40000020024070B5044600257D21C900094893
:106F50000068FEF7CDF8064601F0D4F8002801D00D
:106F6000012504E000222146501E00F033FA284695
:106F700070BD0000880100207047704770B505465D
:106F80003C480078401C3B49087001203A49087091
:106F90003A480088401C394908803948008803F085
:106FA00051F83849C888FEF762FB06463649FEF7B5
:106FB00083F90446354801682046FEF724F9334931
:106FC000086002213248FFF785FF002819D12D49BA
:106FD000C888FEF74CFB06462B49FEF76DF90446C0
:106FE0002C4801682046FEF70EF92A4908602A4914
:106FF00028480068FEF708FC06D828482849C860D9
:1070000002E0002023490860264920480068FEF776
:10701000FBFB03D201202449087002E00020224932
:1070200008701849498F481EFEF716FB044617489A
:1070300001682046FEF7DEFB09D81C4800780028CE
:1070400005D01B48C079012108431949C8710D4971
:10705000488FFEF70CFB04460C4801682046FEF7FB
:10706000C9FB05D211480078002801D004F0AEFE1B
:1070700070BD00007E010020510100206C01002045
:1070800052010020BC0D002000007A448001002045
:1070900000040050780100200000A0400400FA0520
:1070A00000ED00E0000040402E01002066010020BD
:1070B00030120020704710B50446002C01D1012089
:1070C00010BD02212E200155204601F077FD2046FB
:1070D00000F0F4F800212E20015500BF2D200155AD
:1070E00000BF0020ECE77047704710B504462068E9
:1070F0000068C007C00F01214840484000280CD05C
:1071000020688068084048404840002805D0012099
:10711000216848602046FFF731FF2068006802219F
:107120000840400800280BD02068806808404008CC
:10713000002805D00220216848602046FFF71CFF88
:107140002068006804210840800800280BD02068CF
:10715000806808408008002805D004202168486025
:10716000204600F00DF92068006808210840C0089A
:1071700000280BD0206880680840C008002805D08F
:107180000820216848602046FFF794FF20680068C7
:1071900010210840000900280BD0206880680840B2
:1071A0000009002805D01020216848602046FFF71C
:1071B000E4FE2068006820210840400900280BD028
:1071C0002068806808404009002805D020202168F8
:1071D00048602046FFF788FF20680068402108408B
:1071E000800900280BD020688068084080090028AA
:1071F00005D04020216848602046FFF774FF10BD8D
:1072000070B50446002C01D1012070BD60680128D2
:1072100000D100BF26496069884200D000BF2E20FF
:10722000005D002805D100212D200155204600F0E9
:1072300059F802212E2001552068C5686068012890
:1072400003D08905A06A884203D11E2128468843BD
:10725000054617496069884201D01648054016481E
:107260000540A16860680843216A0843616A0843D1
:10727000A16A084305436068012804D00121C905BB
:10728000A06A884203D1E1682069084305430849A0
:107290006069884205D06169A0690843E1690843D3
:1072A00005432068C56001212E2001550020ACE770
:1072B000FFFF00003F1FFFFFF8F119FF10B5044664
:1072C00006492068884208D10548806B4000400884
:1072D000034988630D2000F065F810BD007C004074
:1072E0000010024010B504460949206888420DD1BB
:1072F0000848806B4905084306498863002201213C
:107300000D2000F067F80D2000F058F810BD0000C7
:10731000007C00400010024001460868C0697047C8
:1073200010B5034602242E20C454144800682407D4
:107330002043124C20601868C0680124E4042043F4
:107340001C68E06018688068012420431C68A06005
:1073500018680069012420431C6820611868816155
:107360001868426118680069042420431C68206181
:1073700001242E20C454002010BD00000004014050
:10738000704700000648406B0121084304494863E8
:107390000846806B09040843014988637047000070
:1073A0000010024000BFC206D20E01219140024AE5
:1073B000116000BF7047000080E100E000BFC2061E
:1073C000D20E01219140024A116000BF70470000B7
:1073D00000E100E070B504460D46164629462046F9
:1073E00001F05EFE70BD0000024949688143014A18
:1073F000516070470070004003480068FF21013170
:10740000084301490860704700700040024949681C
:107410000143014A5160704700700040074800680E
:107420000221084305490860054800690421084312
:107430000349086100BF00BF30BF704700700040C3
:1074400000ED00E010B5024600200E4B18688008E1
:1074500080000346134318460A4B18600A4B1B6909
:1074600004242343084C2361012901D130BF02E0E9
:1074700040BF20BF20BF044B1B690424A343024C20
:10748000236110BD0070004000ED00E0F8B5044637
:1074900020212068084020287CD12068084020282E
:1074A00000D100BF00278148806B012109070840F7
:1074B000002805D17D48806B08437C4988630127FB
:1074C0007B480068FF2101310840002816D1784828
:1074D0000068084376490860FFF710FD064606E09D
:1074E000FFF70CFD801B642801D90320F8BD70480C
:1074F0000068FF21013108400028F1D06B48056881
:10750000032109050D4060680840A8420DD009110B
:1075100060680840884208D1644800680121490435
:107520000840884201D10120E0E76048403000690E
:107530000321090408400546002D3DD0606808403D
:10754000A84239D0202120680840202834D157484B
:107550004030006903210904884305465348403000
:1075600000690121C90408435049403108610846B7
:1075700000690121C90488434C494031086108462B
:107580000561801528408915884215D1FFF7B6FCA2
:10759000064608E039E0FFF7B1FC801B4549884208
:1075A00001D90320A2E74148403000690121490286
:1075B0000840400A0028EED000BF00BF03210904A4
:1075C0006068084088420AD1384800680901884349
:1075D000032212056168114008433449086000BF66
:1075E00032484030006903221204616811400843A8
:1075F0002E494031086100BF012F05D12B48806B17
:10760000890588432949886300BF2078C007C00FD7
:10761000002809D025484030C06880088000A16853
:10762000084322494031C8600221206808400228EE
:1076300009D11E484030C0680C218843E1680843E6
:107640001A494031C86004212068084004280AD142
:1076500016484030C06803218902884321690843E5
:1076600012494031C86008212068084008280AD122
:107670000E484030C068032109038843616908430C
:107680000A494031C86080212068084080280AD11A
:1076900006484030C068032189048843A169084333
:1076A00002494031C860002020E70000001002407D
:1076B0000070004088130000F8B504460D46002C09
:1076C00001D10120F8BD79480068C007C00FA84269
:1076D0000ED276480068400840002843734908608D
:1076E00008460068C007C00FA84201D00120E9E7A2
:1076F000022120680840022807D16D48C068F021A7
:107700008843A16808436A49C8602078C007C00F51
:1077100000284CD06068022809D165480068012122
:1077200049040840400C002824D10120CAE76068C1
:10773000032809D15E480068012149060840400E2F
:10774000002817D10120BDE76068012808D15848FA
:10775000006804210840800800280BD10120B1E70F
:1077600053480068012149020840400A002801D11D
:107770000120A7E74E48C068800880006168084380
:107780004B49C860FFF7BAFB0646606802280FD174
:1077900007E0FFF7B3FB801B4649884201D903206D
:1077A00090E74348C0680C2108400828F1D134E034
:1077B000606803280FD107E0FFF7A0FB801B3D495D
:1077C000884201D903207DE73948C0680C21084070
:1077D0000C28F1D121E0606801280FD107E0FFF704
:1077E0008DFB801B3349884201D903206AE730486A
:1077F000C0680C2108400428F1D10EE007E0FFF733
:107800007DFB801B2B49884201D903205AE7284879
:10781000C0680C2108400028F1D124480068C00746
:10782000C00FA8420ED921480068400840002843F4
:107830001E49086008460068C007C00FA84201D072
:1078400001203FE7042120680840042808D1184897
:10785000C068072109028843E16808431449C860E9
:10786000082120680840082809D11148C06807216C
:10787000C90288432169C90008430D49C86000F066
:1078800049F80B49C968F022114009090A4A515CBC
:10789000C8400A4908600020FFF754FB0746002F44
:1078A00001D038460EE700200CE70000002002401F
:1078B00000100240881300004EC00008880100201C
:1078C00001480068704700008801002000B5FFF7FC
:1078D000F7FF0549C968072212021140090A034A45
:1078E000515CC84000BD0000001002405EC00008AE
:1078F00000B5FFF7E5FF0549C9680722D20211402C
:10790000C90A034A515CC84000BD00000010024093
:107910005EC00008FEB52E48C7680C20384000281D
:1079200045D0042804D008280CD00C283ED10BE008
:107930002748006810210840002801D0254C00E0AD
:10794000254C41E0254C3FE00F2080043840800C5E
:1079500023490E5C032080053840800D401C0190B7
:107960001B48C068012109040840002807D01B49B2
:10797000714308460199FDF7BBFB054614E0144826
:10798000006810210840002807D0124971430846BA
:107990000199FDF7ADFB054606E00F497143084626
:1079A0000199FDF7A5FB05462C460DE000BF0848F0
:1079B0004068072149030840400B00900098401C94
:1079C00001218140CC0300BF00BF2046FEBD000066
:1079D0000010024000093D000024F40000127A006B
:1079E00066C00008FEB50446002C01D10120FEBD92
:1079F000F848C6680C210E40C768012109040F40F1
:107A00002078C007C00F002872D0082E04D00C2E9A
:107A10000FD1084687420CD1EE4800680121490485
:107A20000840400C002863D06068002860D1012025
:107A3000DDE700BF012109046068884205D1E548FF
:107A400000680843E349086027E0052109046068ED
:107A500088420ED1DF480068012189040843DD49CE
:107A6000086008460068012109040843D9490860F4
:107A700013E0D8480068012109048843D54908600B
:107A800008460068012109040840009000BFD14861
:107A9000006889008843CF49086000BF60680028FB
:107AA00013D0FFF72BFA054606E0FFF727FA401B35
:107AB000642801D903209AE7C648006801214904D7
:107AC0000840400C0028F0D012E0FFF717FA0546F6
:107AD00006E0FFF713FA401B642801D9032086E76C
:107AE000BC480068012149040840400C0028F0D13E
:107AF00002212068084002287AD1E0680290042E12
:107B000003D00C2E34D1002F32D1B24800680421AA
:107B100008408008002804D00298002801D10120E4
:107B200065E7AC4840681F210902884321690902C2
:107B30000843A8494860084600680921884302991B
:107B40000843A4490860FFF7E5FEA249C968F0228E
:107B500011400909A04A515CC840A04908600020B2
:107B6000FFF7F0F901900198002841D001983EE715
:107B70000298002824D09748006809218843029978
:107B8000084394490860FFF7B9F9054606E0FFF796
:107B9000B5F9401B022801D9032028E78D48006869
:107BA0000421084080080028F1D08A4840681F213D
:107BB000090288432169090208438649486017E0A1
:107BC000844800684008400082490860FFF796F941
:107BD000054606E0FFF792F9401B022801D9032071
:107BE00005E77C4800680421084080080028F1D19E
:107BF000102120680840102867D1002E36D1754822
:107C0000006849010840400A002804D0A069002803
:107C100001D10120EBE66F48406807214903884302
:107C2000216A08436B494860084640680002000A20
:107C3000217F0906084367494860206A400B401CC1
:107C400001218140C8036349C968F0221140090934
:107C5000614A515CC840614908600020FFF772F931
:107C60000190019800284BD00198C0E6A069002837
:107C70002CD058480068FF2101310843554908605D
:107C8000FFF73CF9054606E0FFF738F9401B0228EC
:107C900001D90320ABE64F480068012149020840A2
:107CA000400A0028F0D04B48406807214903884328
:107CB000216A084347494860084640680002000AB4
:107CC000217F090608434349486019E0414800689C
:107CD000FF21013188433F490860FFF70FF905464E
:107CE00006E0FFF70BF9401B022801D903207EE6CE
:107CF00038480068012149020840400A0028F0D1B4
:107D0000082120680840082839D1606900281BD064
:107D1000304840300069012108432E494031086154
:107D2000FFF7ECF8054606E0FFF7E8F8401B0228ED
:107D300001D903205BE62748403000690221084052
:107D400040080028F0D01AE022484030006940087E
:107D50004000204940310861FFF7D0F8054606E0B1
:107D6000FFF7CCF8401B022801D903203FE6194851
:107D7000403000690221084040080028F0D1042169
:107D800020680840042879D1002000901148806BB9
:107D900089060840002806D10E48806B08430D492B
:107DA0008863012000900E480068FF2101310840DF
:107DB00000281ED10A480068084309490860FFF7F7
:107DC0009DF805460EE0FFF799F8401B642809D995
:107DD00003200CE6001002404EC00008880100207D
:107DE0000070004085480068FF21013108400028EC
:107DF000E9D000BFFF210131A068884205D1804849
:107E0000006908437E49086130E0A06800280DD170
:107E10007B480069FF2101318843794908610846A0
:107E2000006909158843764908611FE005210902A8
:107E3000A06888420DD17248006901218902084377
:107E40006F49086108460069891508436C49086153
:107E50000CE06B480069FF210131884368490861E3
:107E600008460069091588436549086100BFA06894
:107E7000002815D0FFF742F8054608E031E0FFF78B
:107E80003DF8401B5F49884201D90320AFE55C48BB
:107E90000069012149020840400A0028EFD013E0A0
:107EA000FFF72CF8054607E0FFF728F8401B554977
:107EB000884201D903209AE551480069012149020D
:107EC0000840400A0028EFD10098012808D14C480A
:107ED0004038806B0121090788434949403988634C
:107EE00000BF606A00284CD00C2E69D0606A02285E
:107EF00048D1434840380068012109068843404979
:107F000040390860FEF7FAFF054606E0FEF7F6FF87
:107F1000401B022801D9032069E539484038006830
:107F2000012149060840400E0028EFD1E16AA06A0D
:107F30000843216B084332494039C968FD221204C5
:107F4000914308432E494039C86008460068012122
:107F5000090608432A4940390860FEF7CFFF054665
:107F600006E0FEF7CBFF401B022801D903203EE5C7
:107F7000234840380068012149060840400E002887
:107F8000EFD038E01E4840380068012109068843D8
:107F90001B4940390860FEF7B1FF054606E0FEF7D1
:107FA000ADFF401B022801D9032020E514484038CA
:107FB0000068012149060840400E0028EFD11AE070
:107FC000606A012800D112E50D484038C7680120D9
:107FD00000043840A16A88420BD10F208004384049
:107FE000E16A884205D1032080053840216B884230
:107FF00001D00120FBE40020F9E400000070004003
:10800000401002408813000010B50446002C01D136
:10801000012010BD606A002800D100BF0021A162CC
:108020005120005D002804D150200155204600F069
:1080300035F802215120015520680068402188430D
:1080400021680860A16860680843E1680843216905
:1080500008436169084301225202A16911400843A3
:10806000E1690843216A0843A16A0843216808605E
:10807000A069000C04210840616A08432168486037
:108080002068C069910088432168C861002060654C
:108090000121512001550020BBE7000010B586B03A
:1080A0000446142101A8FDF796F814492068884277
:1080B00022D11348406B891408431149486300BF1B
:1080C0000846C06A012108430D49C8620846C06AD3
:1080D000C007C00F009000BF00BFE0200190022049
:1080E000029000200390032004900020059001A935
:1080F00005200007FEF7F8FD06B010BD0030014076
:108100000010024070B504462546681E09498842A1
:1081100001D901200CE0681E074948610321081FAE
:1081200000F0BEFF0020044988610720086100209C
:1081300070BD0000FFFFFF0000E000E070477047E7
:10814000FEB504462068C56920680668206887680F
:108150002807000F0190019800280ED12020284008
:1081600000280AD020203040002806D0206E0028A9
:1081700002D02046216E8847FEBD019800287DD0A0
:10818000F807C00F002804D1FF202130304000281C
:10819000F5D0E807C00F00280BD0FF200130304099
:1081A000002806D0012021680862E06F0121084301
:1081B000E0670220284000280AD0F807C00F0028F6
:1081C00006D0022021680862E06F04210843E067BE
:1081D0000420284000280AD0F807C00F002806D045
:1081E000042021680862E06F02210843E06708204C
:1081F000284000280ED020203040002803D1F80766
:10820000C00F002806D0082021680862E06F08210E
:108210000843E067E06F002846D02020284000286F
:1082200009D020203040002805D0206E002802D040
:108230002046216E8847E06F0090206880684021CA
:108240000840402804D0082100980840002826D083
:10825000204602F00EFA206880684021084040283D
:1082600019D120688068884321688860E06E002802
:108270000DD02548E16E8863E06E00E015E0FEF762
:1082800009FB002810D0E06E816B88470CE0204687
:10829000FFF755FF08E02046FFF751FF04E02046B6
:1082A000FFF74DFF0020E06766E70120000528404A
:1082B00000280CD0012080053840002807D001207C
:1082C0000005216808622046FFF738FF54E7802048
:1082D000284000280AD080203040002806D0606E58
:1082E000002802D02046616E884745E7402028409C
:1082F000002807D040203040002803D0204602F05C
:10830000CAF939E700BF37E7B1A5000810B5044640
:10831000002C01D1012010BDA069002800D000E090
:1083200000BF606F002805D1002170200155204654
:1083300000F02CF8242060672068006840084000A6
:1083400021680860204602F00DFA012800D1E2E71A
:10835000606A002802D0204601F09CFF2068406837
:108360000921C902884321684860206880682A2161
:1083700088432168886020680068012108432168DB
:108380000860204601F0FEFFC5E7000010B586B08A
:108390000446142101A8FCF71EFF364920688842D4
:1083A00066D13548406B012189030843324948634F
:1083B00000BF0846C06A012108432F49C862084629
:1083C000C06AC007C00F009000BF00BF032040027A
:1083D00001900220029000200390032004900420CA
:1083E000059001A905200007FEF77EFC23482449DB
:1083F000086003204860002121488160C16080211D
:1084000001610021416181612021C1610902016294
:10841000FEF7F2FA002801D0FDF72EFC00BF184845
:10842000E066846200BF15481438164908600320CE
:1084300048601021134881600021C16080210161E2
:10844000002141618161C1610162FEF7D5FA002816
:1084500001D0FDF711FC00BF0A48A066846200BF8E
:10846000002201211B20FEF7B5FF1B20FEF7A6FF0F
:1084700006B010BD0038014000100240300002403C
:1084800094170020DC17002070B504460D461646F0
:10849000A06F202863D1002D01D0002E01D1012032
:1084A00070BD01210903A068884208D12069002815
:1084B00005D1E807C00F002801D00120F0E700BF78
:1084C0007020005D012801D10220E9E70121702020
:1084D000015500BF6565582006530020E067222043
:1084E000A067E06E002820D01E48E16EC8621E48DA
:1084F000E16E08631D48E16E48630020E16E886309
:108500002368194624313346626DE06EFEF7C8FADF
:1085100000280AD01020E06700BF0021702001551C
:1085200000BF202060670120BAE700BF0021702053
:10853000015500BF20680068FF2101310843216810
:1085400008602068806801210843216888602068ED
:10855000806840210843216888600020A0E702204D
:108560009EE700001BA6000865A60008C9A5000834
:1085700070477047FFB583B004460D461746606FDD
:10858000202875D1002D01D0002F02D1012007B085
:10859000F0BD01210903A068884208D120690028A4
:1085A00005D1E807C00F002801D00120EFE700BF88
:1085B0007020005D012801D10220E8E70121702030
:1085C000015500BF0020E06721206067FEF796FCA0
:1085D0000190502007535220075301210903A0683E
:1085E000884205D12069002802D10026029502E0C8
:1085F0002E460020029021E0069800900022802163
:108600002046019B02F09CFA002801D00320BEE71F
:10861000002E09D102980088C005C00D216888622B
:108620000298801C029003E0307821688862761CF2
:108630005220005B401E81B2522001535220005B49
:108640000028D9D106980090002240212046019BA5
:1086500002F076FA002801D0032098E72020606716
:1086600000BF00217020015500BF00208FE7FFE709
:1086700002208CE7704700BFFEE710B500220421FE
:1086800005200007FEF733FC002208210520000723
:10869000FEF72DFC0A2002F0F9FD0122042105203D
:1086A0000007FEF724FC0A2002F0F0FD002204215E
:1086B00005200007FEF71BFC10BD10B500220421A9
:1086C00005200007FEF713FC012208210520000702
:1086D000FEF70DFC0A2002F0D9FD0122042105203D
:1086E0000007FEF704FC0A2002F0D0FD002204215E
:1086F00005200007FEF7FBFB10BD70B50546002402
:1087000000261EE00022042105200007FEF7EFFBF3
:108710000A2002F0BBFD0122042105200007FEF71C
:10872000E6FB6006040E082105200007FEF7D2FBD9
:10873000002801D0601CC4B2052002F0A7FD701C07
:10874000C6B2082EDEDB002D02D1FFF7B6FF01E036
:10875000FFF793FF204670BD70B504460022042148
:1087600005200007FEF7C3FB00252AE080202040FB
:10877000C011002806D00122082105200007FEF7BD
:10878000B6FB05E00022082105200007FEF7AFFB3D
:108790006006040E0A2002F079FD01220421052062
:1087A0000007FEF7A4FB0A2002F070FD002204215E
:1087B00005200007FEF79BFB0A2002F067FD681CFE
:1087C000C5B2082DD2DB70BD10B5012208210520ED
:1087D0000007FEF78CFB0122042105200007FEF7AD
:1087E00086FB0022082105200007FEF780FB0A20F7
:1087F00002F04CFD0022042105200007FEF777FB64
:1088000010BD10B50022042105200007FEF76FFB04
:108810000022082105200007FEF769FB0A2002F06C
:1088200035FD0122042105200007FEF760FB01222F
:10883000082105200007FEF75AFB0A2002F026FD5A
:1088400010BD10B500240122082105200007FEF705
:108850004EFB062002F01AFD01220421052000072C
:10886000FEF745FB062002F011FD07E0601CC4B2D4
:10887000FA2C03DDFFF7C5FF012010BD08210520FC
:108880000007FEF727FB0028F0D100220421052075
:108890000007FEF72CFB0020EFE7000038B501F0E1
:1088A000A9FD01F0FBFD6E480068C0690221084087
:1088B000002802D06B486C49C860FDF737FB0446BE
:1088C0006A484088002808DD68484088401E81B218
:1088D0006648418001206649087065480078002894
:1088E00006D001280AD0022817D0032822D11BE085
:1088F000012291025F48FEF7FAFA1BE0212C06DA0A
:108900000022012189025B48FEF7F1FA04E001220E
:1089100091025848FEF7EBFA0CE00022012189028F
:108920005448FEF7E4FA05E0012291025148FEF7AF
:10893000DEFA00BF00BF0121C9024E48FEF7CAFAA5
:10894000002828D000204C4908604C4800780028B6
:1089500004D101204949087002F03AF948480078EA
:1089600063280BDD002208214248FEF7C0FA0122ED
:10897000D10305200007FEF7BAFA1BE00122082107
:108980003C48FEF7B4FA00220121C9030520000784
:10899000FEF7ADFA0EE000203849087000220821E9
:1089A0003448FEF7A4FA00220121C903052000077C
:1089B000FEF79DFA2D48808C012820D100253148F2
:1089C000009072B680213048FDF772F90546002DFF
:1089D00005D0022269462C48FDF75CFA054662B6CE
:1089E0002AA002F001FA00212048818403F09EFAB7
:1089F000642002F041FC1B481B49C86000BF1B48B3
:108A0000408C01280ED100211848418400201749CC
:108A10004039088003F08AFA642002F02DFC1148E6
:108A20001149C8601148008C01280AD100210F4863
:108A3000018403F07BFA642002F01EFC09480A4915
:108A4000C8600A48403800881449884204D1074861
:108A50004038C088002802D102480349C86038BDA8
:108A6000141700200400FA0500ED00E0FC0D0020C2
:108A70003601002000040050800100206801002021
:108A800050010020AAAA0000384A0008BDF8C8EB2F
:108A9000C9FDBCB6C4A3CABD0D0A0000AA5500009A
:108AA00008B53721202000F077F80321212000F0BD
:108AB00073F84021222000F06FF80821232000F0F5
:108AC0006BF8AA21302000F067F802200B490887D4
:108AD0000846008FC1B2322000F05EF80121332039
:108AE00000F05AF85F21202000F056F8684600F0A8
:108AF00007F80A2002F0CAFB08BD0000BC0D0020E8
:108B000010B5044621460F2000F023F8002800D1BC
:108B100010BD0120FCE770B504460025FFF754FEA8
:108B20003220FFF719FEFFF78CFEE0B2FFF714FECC
:108B3000FFF787FEFFF748FE3320FFF70DFEFFF734
:108B400080FE0020FFF7D9FD0546FFF75AFE2846B4
:108B500070BD70B505460C462846FFF7DCFF207057
:108B6000012070BD70B504460D46FFF72DFE322082
:108B7000FFF7F2FDFFF765FEE0B2FFF7EDFDFFF74F
:108B800060FE2846FFF7E8FDFFF75BFEFFF739FEC2
:108B90000A2002F07BFB70BD70B504460D462946E5
:108BA0002046FFF7DFFF012070BD000010B502482E
:108BB000FEF79BFA10BD00008C160020F0B585B0C2
:108BC00004460020039072B64F49206840180028E0
:108BD00006D14E48C068032189040840039000E094
:108BE00000BF00BF2068806802902068C0680190C4
:108BF0002068456920688669434920684018002834
:108C00000DD142484038806A490508433F49403900
:108C100088620846806A40004008886200E000BF21
:108C200000BF002D01D1002E5FD0374920684018C9
:108C3000002807D13548C068032189048843334997
:108C4000C86000E000BF00BF002D1DD02068006993
:108C5000012108432168086120684561FEF74EF94B
:108C6000074600BFFEF74AF9C01B00902068006865
:108C700008210840082804D07D21C90000988842B6
:108C8000F0D9082021684860002E1DD020680069B6
:108C9000012108432168086120688661FEF72EF9EA
:108CA000074600BFFEF72AF9C01B00902068006845
:108CB00010210840102804D07D21C9000098884266
:108CC000F0D91020216848600F492068401800281A
:108CD00009D10E48C06803218904884303990843D9
:108CE0000A49C86000E000BF00BF20680069400872
:108CF0004000216808610298216888600198216815
:108D0000C86062B605B0F0BD0084FFBF40100240ED
:108D10001CB50020009001901E481F4908600021EA
:108D20001D48C163012080071B49486000211A4883
:108D3000816007218163012101610021C160001D63
:108D400001774177001F8162FF21C231416200211A
:108D500024300172042124384161002101638161C2
:108D60004163C161FDF796FB002801D0FCF784FF49
:108D70000A4800908013019069460748FDF7FEFA03
:108D8000002801D0FCF778FF00210348FDF788FA9E
:108D90001CBD000000240140301600200200000429
:108DA00008B500BF0A48006B012108430849086361
:108DB0000846006BC007C00F009000BF00BF002234
:108DC00001210A20FEF706FB0A20FEF7F7FA08BD8C
:108DD0000010024000B587B0142102A8FCF7FBF98F
:108DE00000BF6548C06A042108436349C862084659
:108DF000C06A04210840019000BF00BF00BF5E4868
:108E0000C06A802108435C49C8620846C06A802164
:108E10000840019000BF00BF00BF5748C06A012151
:108E200008435549C8620846C06AC007C00F019090
:108E300000BF00BF00BF0846C06A022108434E4978
:108E4000C8620846C06A02210840019000BF00BF06
:108E500001221C2105200007FEF749F8012247499D
:108E60004748FEF744F8002246494548FEF73FF8D8
:108E700000229121090205200007FEF738F80120A1
:108E80000290414803900020049002A905200007A9
:108E9000FDF72AFF02200290032003900020049097
:108EA00002A905200007FDF71FFF0C2002901120EA
:108EB0000390002004900320059002A905200007DC
:108EC000FDF712FF10200290012003900020049073
:108ED0000220059002A905200007FDF705FF0120EB
:108EE00002901120039000200490059002A92448CC
:108EF000FDF7FAFE0220029024480390012004901E
:108F000002A91F48FDF7F0FE2148029001200390BE
:108F100000200490059002A91948FDF7E5FE012004
:108F2000C0020290002003900220049002A914487D
:108F3000FDF7DAFE9120000202900120039000204C
:108F40000490059002A905200007FDF7CDFE8020C2
:108F50000290002003900120049002A90848FDF728
:108F6000C3FE002201210520FEF734FA0520FEF79A
:108F700025FA07B000BD0000001002400106000005
:108F80000004005008300000000011100000211003
:108F90000836000010B50A480A49086000204860F9
:108FA0000021084881600849416100210162416255
:108FB0008162FEF725F9002801D0FCF75DFE10BDA7
:108FC000007C00408C160020FFFF000010B5124806
:108FD00012490860FF200530486000210F48816079
:108FE000C160016141610121490281610021C161CA
:108FF0000162416281620721C162FFF705F8002822
:1090000001D0FCF739FE054800680068402108439C
:1090100002490968086010BD00300140BC160020FC
:1090200000B585B014216846FCF7D5F819481A49EF
:109030000860E12040024860002117488160C1605B
:1090400001610C21416100218161C1610162302017
:1090500011494862012109030F4881634900C16336
:10906000FFF754F9002801D0FCF706FE012080022A
:109070000090022001900120029003200390042020
:109080000490694605200007FDF72EFE01F09AFDC9
:1090900005B000BD003801401417002070470000E3
:1090A00010B5002819DA1A4A03071B0F083B9B0862
:1090B0009B00D2588307DC0EFF23A3409A438B0703
:1090C0001B0E8407E40EA3401A43114B0407240F20
:1090D000083CA408A4001A5118E00E4A03231B02FE
:1090E000D21883089B00D2588307DC0EFF23A340CD
:1090F0009A438B071B0E8407E40EA3401A43054BCB
:10910000032424021B198408A4001A5110BD000076
:109110001CED00E000E100E000BF00BF00BFBFF3B6
:109120004F8F00BF00BF00BF06480749C86000BF9F
:1091300000BF00BFBFF34F8F00BF00BF00BF00BF25
:1091400000BFFDE70400FA0500ED00E0F0B593B0C4
:1091500000200E90962002F003FC4B20C00002F08D
:109160001BFC0020FE490870FE4800780C2802DB3A
:109170000B20FC4908700122510205200007FDF771
:10918000B6FE0020F8490870F8490870F8480078E1
:10919000F84908710221F848FDF79CFE002801D12A
:1091A000012000E00020F549097849000843F14911
:1091B000C871F34801780068401CF14A1060C8B2D9
:1091C000EC49C870EF4800788872EE480078420099
:1091D000ED49E8480B30FBF7E5FF0620E54948720A
:1091E0000846EA490A78427049788170E549097869
:1091F000490008460D300022DE4902F0CFFCE1496B
:109200000978490008460D30002102F0DBFC0220FD
:1092100002F000FC0020D749C871DD490870DD4923
:1092200008700120DC4908700020DC490870DC4827
:10923000FEF772F8DB4908800020CB490870D1485E
:109240000078FCF714FA0746FCF790FA0022D64B98
:1092500005910490FCF720F90791069001F0A8FF12
:109260000022D24B09910890FCF764F80B910A9008
:10927000FCF75EFAC0B20D900D984001C94909880B
:109280004018CB490880084600880121C90388425C
:1092900004DBC7480088401AC5490880C548C6494C
:1092A0000860C6480078401CC4490870BC48FEF7F6
:1092B00033F8C34908807AE2B948FEF72DF8C0496F
:1092C000088033E0B348007800281BD002F004FB8C
:1092D000109012991098884214D9119910988842C8
:1092E00010D202F085F90020AB490870304602F038
:1092F0002FFB012002F08EFBB24908700020A54927
:1093000008701DE0A648FEF707F8AD49088008463A
:109310000088A7490988884208DBA9480088A44931
:109320000988A94A8918884200DA09E000210F203B
:1093300002F06EFAA5490860A54908400028C1D08E
:1093400000BFA2480068401C002801D1FFF7E4FEDE
:109350009E48006801218903084000287ED08122B0
:10936000D20100210F2002F0D2FB0021102002F0D8
:109370004FFA4006400E0F90002296480F9902F0D7
:1093800097FA002002F008FB002002F0B4FA91489E
:10939000407A07288FD102228F498E48401DFBF763
:1093A00025FF002887D102F06AFC8C4A03C202F034
:1093B0004FFC8B4A03C26C480078401C6A49087015
:1093C0008448427808A90A74817808A841746846DC
:1093D000008E6E49098888427ED182497D48C089C5
:1093E000088081487B49098A01806D48FDF794FF18
:1093F000734908807C480088FF30C3307A49088070
:10940000084600887949884212DD77480088401A6A
:109410007549088073480088401C724908800846D6
:10942000008872490B31884202DB00206D490880B8
:109430006F49684842890A808089488008460068E8
:109440005D4908606348C07C0007000F032807D00F
:109450006048C07C0007000F444900E09BE10870B1
:109460005C48C07C001163490870002053490870B3
:109470000120484908705049564842890A8080892D
:10948000488040480078FF2191314843FF30FF3049
:10949000FF30F5300004C117514B0CCB80185941F7
:1094A0000906060A0E435448301A12901920800209
:1094B000301811907108490000200A0E0002104374
:1094C0000B02002211469A1848414C490A60486034
:1094D00042480CC8274800E0FBE00A3002F09EFB3F
:1094E0003F480CC82348163002F098FB43480CC88C
:1094F0002048123002F092FB08201E4948723D4875
:109500000078002817D0022233493248401DFBF76B
:109510006DFE00280FD101201D4908701549C87142
:109520000F981638364908700846027829491431D0
:109530003448FBF737FE13490978890008461C3088
:1095400000220C4902F02AFB0E49097889000846DE
:109550001C30002102F036FB01201049087053E056
:10956000E90000202A010020090100203601002026
:109570005001002030120020000400502E01002075
:109580006C000020280100202A1400200201002085
:109590002C0100201C0100201E0100201D010020C4
:1095A0008C160020220100200000E03F000008404F
:1095B00024010020A08601000401002019010020E0
:1095C00020010020E8000020983A000070000020F0
:1095D00000D02724801200204401002078000020C1
:1095E000800000204C010020F4000020E703000070
:1095F000F8000020370100200052030088000020FE
:109600002D010020F81400200422F049F048FBF757
:10961000C9FDF04800887D21C9004843EE4909880A
:109620004018EE490860EE480078EE490870EE49AF
:10963000C888FCF71CF80990E6480088FCF717F882
:1096400008900999FBF738FE7F21C9050A90FBF7BE
:10965000DAFD0B90FCF734F8E1490880E148007826
:10966000401E0988884202D10120E0490870D9488B
:109670000088DF490880DF490020085EFBF7FEFF15
:1096800009910890DC480088FCF70CF8DB4ADC4BB9
:1096900001910090FBF700FF05910490CF4800680E
:1096A000FBF7ECFF03910290059B049AFBF7E6FEA3
:1096B00007910690099B089AFBF73CFE0B910A90D4
:1096C000FCF712F8CF490860CF48008800F0BAFCD8
:1096D00060E06846008EFCF70BFC07460321CB4A8E
:1096E000D155CB49B948401E42890A8080894880BB
:1096F00008460168B800C74A1150B448401EC07CF3
:109700000007000FC449097888420BDDAF48401EAE
:10971000C07C0007000F032804D0AC48401EC07C6A
:10972000BD490870BD480078002817D00222BC4906
:10973000A648001DFBF75AFD00280FD10120B949AA
:109740000870B949C8710F981638B84908700846AA
:1097500002789E491331B648FBF724FD781C80003F
:109760001630B14940180B90B2480CC80B9802F063
:1097700055FAB1490978890008461C300022AA49E7
:1097800002F00CFAAC490978890008461C30002127
:1097900002F018FA0BE0A94A00210F2002F0B7F9F5
:1097A000A7480078002802D0002002F0A4F89248D0
:1097B0000088A4490988884200DA7DE58E4800883F
:1097C000A0490988A04A89188842F6DC9B4A0021F2
:1097D0000F2002F09CF900248C480078002818D152
:1097E0007B480068FCF76CFC984908800888098869
:1097F000491E964B198096490988FBF78FFC9548BE
:109800000088414388B2804908800846008800F0FB
:1098100019FC002090490870002523E07B48405D3A
:1098200000281DDD8C480078401C8B490870774863
:10983000405DA100894A505068008949085A61007A
:10984000884A5052A80073490A582146601CC4B285
:10985000880085490A506D48405D401E6B49485557
:10986000681CC5B2744800788542D7DB7F48007811
:10987000032803DA7848007877490870764800783A
:109880007B49087000253FE0002436E0A0007649BF
:109890000958601C8000744A105881422BDDA200D8
:1098A000714B995862006F4B985AAA006B4B9A58AB
:1098B0000C92621C92006C4B9A58A3006A4FFA50AB
:1098C000621C5200674B9A5A6300664FFA52621C40
:1098D0009200624B9A58A300604FFA50621C9200AB
:1098E000614B9950621C52005E4B9852631C9B0066
:1098F0000C9AFA5000BF601CC4B25D480078401E4C
:10990000A042C3DC681CC5B259480078401EA8427A
:10991000BADC55480168574800683238814205DA98
:1099200055480078401C5449087002E00020524914
:10993000087051480078032806DD4A4800884F49DE
:10994000088001204E4908704E480078032802DD47
:1099500000204B490870002505E04B48A9002D4A1E
:109960005050681CC5B20C2DF7DB2E48007800283B
:109970001CD000200C9000270B902D4800780B90F5
:109980002B48477880780C900B9802280DD1164907
:10999000C8192749C91C0C9AFBF704FC02F0C6FA47
:1099A000642001F069FCFFF7B7FB00BF234A803257
:1099B00000210F2002F0ABF800220121490205200E
:1099C0000007FDF794FA13B0F0BD000081120020EB
:1099D000300100204C010020F40000200C01002088
:1099E0006C0100202B010020BC0D00201D01002077
:1099F000260100203401002020010020F853E3A5B7
:109A00009B843E401401002052010020EC140020F1
:109A1000F80000205C1400203601002037010020EF
:109A2000440100202C010020301200202D010020D4
:109A3000F8140020800000202801002000D02724F6
:109A40001E01002024010020983A0000FC000020A4
:109A500058010020560100202A010020BC140020DB
:109A60002A140020421400208C1400200901002038
:109A700029010020040100203A01002002010020F9
:109A80006000002019010020FFFF01007047000066
:109A9000FEB5AC4802900020C043019000279620FC
:109AA00001F05EFF4B20C00001F076FF0020A649C8
:109AB0000870002622E1A548867300220146142082
:109AC00002F06CF80021142002F07CF8022001F072
:109AD000A1FF00BF00210F2001F09AFE9C49086001
:109AE0009C4908400028F5D099480068401C00288F
:109AF00001D1FFF711FB9648006801218903084056
:109B000000287DD08122D20100210F2001F0FFFF2B
:109B10000021102001F07CFE45066D0E2946002232
:109B20008D4801F0C5FE8C48407A022869D1022296
:109B30008A498948401DFBF759FB0028F6D102F0FD
:109B40009EF8874A03C202F083F8864A03C2002FB8
:109B50002BD1012784498048C089088083487E49E9
:109B6000098A01808248FDF7D7FB824908807F4837
:109B70000088FF30C3307D490880084600887E4950
:109B8000884212DD79480088401A78490880764872
:109B90000088401C744908800846008876490B31CB
:109BA000884202DB0020704908806B484289694680
:109BB0000A808089488004226749491C6F48FBF766
:109BC000F1FA684803684068FF22520400219A189D
:109BD00048410106140A0C43204601F0B9FE610811
:109BE000490000200A0E000210430B020022114619
:109BF0009A18484162490A60486059480CC801E017
:109C000072E06DE05D48093002F008F855480CC874
:109C10005A480D3002F002F859480CC85748113024
:109C200001F0FCFF00225549491E3C2001F0B6FF1F
:109C300000213C2001F0C6FF012001F0EBFE51495C
:109C4000087041480078401C3F4908700121C90351
:109C500005200007FCF762F94B480068FCF730FA72
:109C60004A49088008880988491E484B1980484994
:109C70000988FBF753FA47480088414388B24649B0
:109C800008800846008800F0DDF9009902988142BA
:109C900010DA009800280DD004222F49491C01A891
:109CA000FBF780FA01203D49087005203C49087007
:109CB0000098029033480078002808D100BF0021A6
:109CC0000F2001F0A5FD802108400028F7D0802258
:109CD00000210F2001F01BFF0020324908700BE02B
:109CE00001203049087007E02F4A00210F2001F0C1
:109CF0000EFF01202B490870701CC6B2032E00DA3B
:109D0000D9E6002F1AD121480088401E1F4908803B
:109D100008460088002805D0084600881C490988A4
:109D2000884203DD1A4800881849088017480088CF
:109D3000401E184909884843174908801B49019863
:109D40000880FEBD3F420F00E9000020BC1100204A
:109D50007000002000D02724801200204401002041
:109D600078000020800000204C010020F40000203A
:109D70008C16002020010020E7030000DF110020E6
:109D800088000020E800002030010020FC000020B6
:109D900058010020560100205201002060000020E0
:109DA00008010020BC0000200090272402010020B0
:109DB000F8B546484649086002F044F84548464927
:109DC00048800846C088002801D16420C8804348E4
:109DD0000078432802DD4320404908703F4800785E
:109DE000002802DA00203D4908703B48C08E3B49FC
:109DF00008703948C08F3A4908703748808F394910
:109E000008703548807A3849087033488088374967
:109E100008600520364908802F49C88834490988D8
:109E2000FBF77CF9334908802B4988883149098838
:109E3000FBF774F92E480088414388B22E49088008
:109E400009887D22D20051430846FBF717FC0446DF
:109E50002A4A2B4BFBF788FB0646FBF769FC29498E
:109E6000088025480088284908801B48C1887D2033
:109E7000C000FBF753F9254908801748C1887D20A9
:109E8000C000FBF74BF922490880012021490880D6
:109E9000FCF74CF8204908801A4802881F492048DE
:109EA000FDF73EFA002801D0FBF7E6FE0F480168F7
:109EB0001CA000F099FF0848C1881EA000F094FF84
:109EC0000548018920A000F08FFFF8BD0DAC000807
:109ED0004800002001020000BC0D0020010000200D
:109EE00066010020670100204F010020440100208E
:109EF000560100205801002052010020F853E3A52C
:109F00009B843E405E010020620100206001002031
:109F10006A0100206C01002064010020FF7F000026
:109F20008C160020B1EAC7A949443A202564202EA6
:109F30000D0A0000CDA8D1B6BCE4B8F43A202564DF
:109F4000206D732E0D0A0000B5A5B4CECDA8D1B6F4
:109F5000BBF9D5BECAFDC1BF3A202564B8F62E0DA7
:109F60000A00000000B585B014216846FBF733F9FC
:109F700000220121C9031048FCF7B9FF0120C003EA
:109F800000900120019000200290039069460A4849
:109F9000FCF7AAFE0120C0030090032001900020DE
:109FA0000290039069460448FCF79EFE022001F0EF
:109FB00063F905B000BD00000004005070470000C8
:109FC00038B504460D460020009055201B49087006
:109FD000AA20487003208870601DC8700320087193
:109FE0000846457184716800154A81182246134855
:109FF000C01DFBF7D7F8002008E0811C0F4A525C17
:10A000006946098851188AB20092401C611D884235
:10A01000F3DB0A48801CFBF77BFD0090E01D07493D
:10A0200041186846007808706846407848702146B4
:10A030000931024800F048FB38BD0000CC15002073
:10A04000BC0D0020F0B585B005461A4800881A49B5
:10A050000988884206DB1748008817490988401A92
:10A06000144908801548C08812490988484347198F
:10A070007D21C9004F43124800683E1A3046FBF765
:10A08000FDFA104A104B01910090FBF76DFA039115
:10A090000290FBF729FB04460C498C4201DD08467F
:10A0A000241A002C01DA0948241809480068446180
:10A0B00005B0F0BD6C0100206A010020BC0D00203D
:10A0C00014010020F853E3A59B843E40FF7F00006D
:10A0D0008C16002001460020054A126890B2054AFD
:10A0E000104002460A431046014A106070470000C3
:10A0F00000300140C7FF000010B5FCF705FF10BDA0
:10A1000000B599B034210CA8FBF765F8142107A815
:10A11000FBF761F81C216846FBF75DF824480068EE
:10A120000321C90288430121C9024018204908605F
:10A13000FDF762F91F4800690321C90288431D49E0
:10A14000086106200C9088150E9001200F901020B9
:10A15000109002201590002116914104179141059D
:10A1600018910CA8FDF73EFC002801D0FBF784FDF8
:10A170000F20079003200890002009900A900B9070
:10A18000012107A8FDF798FA002801D0FBF774FD1C
:10A1900081200090002002900320800406906846F1
:10A1A000FDF774F9002801D0FBF766FD19B000BD7A
:10A1B000007000404010024015480068FF21013146
:10A1C0000843134908600846C0681249084010490E
:10A1D000C86008460068104908400D4908600846F4
:10A1E00080684008400088600846006801218904B2
:10A1F0008843074908600846C068FD210904884370
:10A200000349C86000200861044805498860704718
:10A21000001002400C40FF88F6FFF6FE00500008D8
:10A2200000ED00E010B501F00DFB044602E001F086
:10A2300009FB044613488442F9D1002012490880E2
:10A2400012480078002804D0012805D0022814D133
:10A2500010E0FFF71DFC10E00D480078401E0C498F
:10A260000870FBF785FE0A480078002801D10749ED
:10A27000087002E0FEF76AFF00BF00BF01F09CF922
:10A2800010BD00003001CADEE600002060000020A2
:10A2900008010020818CC907C90F002908D0016876
:10A2A0004968012252049143826A11430268516055
:10A2B0000222416A1140022907D101684968D2038C
:10A2C0009143C26A1143026851600422416A1140FD
:10A2D000042907D10168496812049143026B1143B4
:10A2E000026851600822416A1140082907D10168BB
:10A2F000496812039143426B114302685160102276
:10A30000416A1140102907D10168896812029143FE
:10A31000826B1143026891602022416A114020291A
:10A3200007D10168896812029143C26B1143026828
:10A3300091604022416A1140402915D10168496865
:10A3400092039143026C114302685160012212058D
:10A35000016C914208D1016849680322520591437A
:10A36000426C1143026851608022416A1140802989
:10A3700007D10168496812039143826C1143026856
:10A380005160704738B504460020E067FCF7B6FD21
:10A390000546206800680821084008280BD11448A9
:10A3A0002B46002289040090204600F0C9FB0028BB
:10A3B00001D0032038BD206800680421084004282B
:10A3C0000BD10B482B46002209050090204600F0D7
:10A3D000B7FB002801D00320ECE720206067A067CE
:10A3E00000BF00217020015500BF0020E2E70000FF
:10A3F000FFFFFF0170B50025C82420480078002821
:10A4000000D070BD1E480078002800D0F9E7012078
:10A410001B4908701B48406B002801D10870F0E709
:10A420001848406BC8210D1A1CE01749174A1268DA
:10A43000885C174909688847164800880A214843FC
:10A440001549088011480068401C104908600846FA
:10A450000068C82801DB002008600A48406BC8215A
:10A460000D1A641E09480068A84201D0002CDCDCEB
:10A4700000200349087000BFC3E70000420000202D
:10A480004400002000000240F40C002038000020AE
:10A4900048000020600100207401002010B53A48F7
:10A4A0000078002803D139480078002800D010BD7A
:10A4B0000120364908703648C069802108400028CC
:10A4C00002D132490870F2E7324900200856324979
:10A4D00000228A56904215D12D48C069402108407B
:10A4E00000280BD02D480078002807D000202B49E9
:10A4F00008702B480088401C294908800020234907
:10A500000870D4E725480078002805D101202349A8
:10A5100008700A2000F0BAFE1F4900200856CC211E
:10A52000484320494018001D1F490968405C1849EC
:10A5300088621D480068401C1B49086016490020BD
:10A540000856CC21484317490858174909688842DA
:10A5500014DC0020144908600F480078401C40B209
:10A560000D490870084600780E2801D100200870B7
:10A570000E480078401C40B20C4908700020034986
:10A58000087000BF93E70000420000204300002055
:10A590000038014035000020340000204500002034
:10A5A00052000020CC01002058000020360000207E
:10A5B00070B50546AC6A00215A2001535220015360
:10A5C0002046FDF7BCFD70BDF8B50546AC6A666F68
:10A5D000A76F2068806880210840802807D1212E3D
:10A5E00005D1002152200153204600F064F8206874
:10A5F000806840210840402807D1222F05D1002142
:10A600005A200153204600F034F8E06F102108432F
:10A61000E0672046FDF793FDF8BD70B50546AC6ACE
:10A620002868006820210840002817D100215A20FE
:10A63000015320680068FF210131884321680860C8
:10A640002068806840084000216888602068806831
:10A6500040218843216888602020A0672046FDF7BC
:10A6600087FF70BD70B50446A56A2846FDF781FFD7
:10A6700070BD01680968FF222132914302681160B0
:10A680000168896849084900026891602021816752
:10A6900000210166704710B504462068006840211B
:10A6A000884321680860202060670020606620469B
:10A6B000FDF7E0FF10BD01680968C0229143026800
:10A6C000116020214167704770B505460C4620484F
:10A6D0000078002803D11F480078002800D070BD02
:10A6E00001201B490870C82C04DC1B48002141567E
:10A6F000002903DC002016490870F0E71749002004
:10A700000856CC21484316490C50144A0021515692
:10A71000CC225143124A8918081D22462946FAF7CD
:10A7200041FD0E480078401C40B20C4908700846B4
:10A7300000780E2801D10020087007480078401EDC
:10A7400040B20549087000200149087000BFC6E703
:10A750004200002043000020360000203500002089
:10A76000CC010020F0B587B00446102004900025ED
:10A77000002003900026E7492068884200D100E0CD
:10A7800000BF2169A068084361690843E169084383
:10A79000074620680068E04908403843216808609F
:10A7A00020684068032109038843E1680843216861
:10A7B0004860A769D7492068884201D0206A0743CA
:10A7C000206880680B21090288433843216888602B
:10A7D00000BFD249206888421CD1D148C068800798
:10A7E000800F002806D001280AD0022805D00328AF
:10A7F0000CD108E0012004900BE00220049008E056
:10A800000420049005E00820049002E01020049049
:10A8100000BF46E0C349206888421CD1C048C068D8
:10A820000C210840002806D004280AD0082805D0AA
:10A830000C280CD108E0002004900BE002200490CA
:10A8400008E00420049005E00820049002E01020B5
:10A85000049000BF25E0AF49206888421FD1B0486E
:10A86000C068032189020840002808D0012189021C
:10A87000401A0AD0401A05D0401A0CD108E0002036
:10A8800004900BE00220049008E00420049005E00E
:10A890000820049002E01020049000BF01E0102086
:10A8A000049000BF9B492068884256D10498042830
:10A8B0001AD004DC002807D002281CD108E00828A0
:10A8C00016D0102817D117E0FDF700F8064616E05D
:10A8D000934840380068102108400009002801D042
:10A8E000914E00E0914E0AE0FDF714F8064606E0AE
:10A8F0000126F60303E000BF0120039000BF00BF64
:10A90000002E0AD0606841004018B04203D8606849
:10A910000003B04202D201200390F4E0606802908C
:10A920003046FF21013100F086FA626852080023A8
:10A930008018594101910090029AFAF703FC0546EC
:10A9400003200002854205D37948854202D8206859
:10A95000C560D8E001200390D5E00121C903E0697A
:10A9600088426FD1049804283CD006DC002809D026
:10A97000012813D002284AD11CE008283ED0102814
:10A9800045D145E0FCF7A2FF400061684908401846
:10A9900002906168FAF7ACFB85B23CE0FCF7A8FFD7
:10A9A000400061684908401802906168FAF7A0FB0E
:10A9B00085B230E05A48403800681021084000094C
:10A9C000002807D061684A085A4BD018FAF790FB64
:10A9D00085B206E061684A08574BD018FAF788FB41
:10A9E00085B218E0FCF796FF4000616849084018FE
:10A9F00002906168FAF77CFB85B20CE061684A0856
:10AA000001231B04D018FAF773FB85B203E000BFE3
:10AA10000120039000BF00BF102D0FD3474885428F
:10AA20000CD846480F38284005902807400F059954
:10AA30000843059005982168C86064E001200390F0
:10AA400061E0FFE7049804283AD006DC002809D02A
:10AA5000012812D0022847D11AE008283BD010283C
:10AA600042D142E0FCF732FF616849084018029089
:10AA70006168FAF73DFB85B23AE0FCF739FF61689F
:10AA80004908401802906168FAF732FB85B22FE05E
:10AA9000234840380068102108400009002807D0EA
:10AAA00061684A08204BD018FAF722FB85B206E00D
:10AAB00061684A081D4BD018FAF71AFB85B217E0F7
:10AAC000FCF728FF61684908401802906168FAF7AE
:10AAD0000FFB85B20CE061684A080123DB03D01844
:10AAE000FAF706FB85B203E000BF0120039000BF28
:10AAF00000BF102D05D31148854202D82068C560DB
:10AB000001E001200390002020666066039807B0F2
:10AB1000F0BD000000480040F369FFEF003801403D
:10AB2000401002400044004000093D000024F400B1
:10AB3000FFFF0F0000127A000048E801FFFF00004D
:10AB4000FFB581B004460D4617460A9E22E0701CF0
:10AB500000281FD0FCF7D2F90499401AB04201D85E
:10AB6000002E17D120680068FF21A1318843216899
:10AB700008602068806840084000216888602020C4
:10AB80006067A06700BF00217020015500BF03204F
:10AB900005B0F0BD2068C0692840A84201D101205D
:10ABA00000E00020B842D2D00020F1E710B510201C
:10ABB0000349096808620248FDF7C2FA10BD0000A7
:10ABC000141700200D20014908707047360000203E
:10ABD00010B50A4800880A21484309490880FEF751
:10ABE000DFF8FEF71DFAC82206490748FDF74CFCBE
:10ABF000002801D0FBF740F810BD000060010020E4
:10AC000074010020F40C00201417002070B50446D5
:10AC100000256A480078082865D100BF002004E0BC
:10AC20006749095C49198DB2401C66490978491F7A
:10AC30008142F5DC64480078281885B261480078C4
:10AC4000281885B261480078281885B260480078D5
:10AC5000281885B25F480078281885B26019C007A7
:10AC6000C00F002835D058480078012827D0022886
:10AC70002DD15949554A1278881855490A785049B2
:10AC8000FAF790FA01F052F9642000F0F5FA00BFEB
:10AC900000BF00BF00BF00BFBFF34F8F00BF00BFAA
:10ACA00000BF4E484E49C86000BF00BF00BFBFF3A1
:10ACB0004F8F00BF00BF00BF00BF00BFFDE743488C
:10ACC0000078411042480078FFF77AF900E000BFB1
:10ACD00000BF0020394908703C49087039490870A4
:10ACE0004049087068E035480078072812D1344898
:10ACF0003C49097844543B480078401C3949087065
:10AD000030480078401F0978884255D108202B49E7
:10AD1000087051E029480078062805D12C480470B5
:10AD200007202649087047E024480078052805D107
:10AD3000264804700620214908703DE01F4800782D
:10AD4000042805D12048047005201C49087033E010
:10AD50001A480078032808D11A48047000201B49BB
:10AD6000087004201549087026E01448007800286F
:10AD700005D1552C03D10120104908701CE00F4863
:10AD80000078012805D1AA2C03D102200B490870B4
:10AD900012E00A480078022807D1032C05D10320CD
:10ADA000064908700B48047006E00020034908704B
:10ADB000064908700349087070BD00003B0100207F
:10ADC000681500203D010020400100203E010020C8
:10ADD0003C0100203F010020BC0D00200400FA05CA
:10ADE00000ED00E0410100200FB410B503A9044BB1
:10ADF000044A029800F034F910BC08BC04B01847AB
:10AE000039BC00088C0100202021020C01D0102147
:10AE10001046020A01D010460839020901D0104636
:10AE2000091F820801D01046891E420801D0881EE1
:10AE30007047081A7047F8B582B28BB2040C0D0C3B
:10AE400010465843002126465E43370C36048019CD
:10AE5000794116466E43370C3604801979412646EF
:10AE60006E438919F8BD30B47446641E2578641C9D
:10AE7000AB4204D3635D5B00E31830BC18471D464A
:10AE8000F8E702E008C8121F08C1002AFAD170478B
:10AE90007047002001E001C1121F002AFBD170475A
:10AEA00008B5002100916B46012202212C2000F000
:10AEB00043FE022100916B4601222C2000F03CFE53
:10AEC00008BD000038B504466D2000906B46012295
:10AED00008492E2000F030FE002C05D0064A074914
:10AEE0002E2000F003FE04E0054A04492E2000F065
:10AEF000FDFD38BD0608000007060000061800002A
:10AF00000716000038B504466B46022200213620A1
:10AF100000F09EFC2300FFF7A6FF0E11081A545400
:10AF20005454233154543D444B540021684601701D
:10AF30004078FE2108406946487043E06946087839
:10AF4000FC21084001210843694608703AE069463F
:10AF50000878FC210840022108436946087031E066
:10AF600068460078B32108404821014368460170D3
:10AF70004078802108436946487023E0684601789C
:10AF8000B32001406846017040784106490E68468A
:10AF9000417017E0694648780221084369464870C5
:10AFA00010E069464878FD2108406946487009E08C
:10AFB00069460878CF210840202108436946087077
:10AFC00000E000BF00BF6B4601220021362000F0E8
:10AFD000B3FD00AB013301221146362000F0ACFD79
:10AFE00038BD08B5032168464170012101706B46E8
:10AFF00002220021362000F09FFD0122D20306210B
:10B000002D2000F073FD012000F036F90120FFF73C
:10B0100079FF08BD38B504462004010E684641702A
:10B0200004706B46022204212D2000F085FD0321CF
:10B03000684601706B46012206212D2000F07CFD40
:10B040000021684601706B46012206212D2000F088
:10B0500073FD0A212D2000F0DBFB0546284638BD94
:10B06000FFB58DB00446002506E025280AD0109AC9
:10B070000F999047641C6D1C20780028F5D1284654
:10B0800011B0F0BD00270121484A009700E00743B6
:10B09000641C23780846203B98401042F7D1207862
:10B0A0002E2817D1042007436078641C2A280CD16D
:10B0B0000E98641C02C800910E900BE000990A22C1
:10B0C000514330394018641C0090207801463039D3
:10B0D0000929F3D920780028D1D0642808D069281C
:10B0E00006D075281ED0109A0F9990476D1C5BE012
:10B0F0000A200E99019001C90E91002802DA4042FF
:10B100002D2102E0390504D52B216A461172012157
:10B1100003E0F90704D02021F7E70BAE0B910DE017
:10B120000021FAE70A200E99019001C90E91F7E774
:10B130000199F9F7DDFF3031761E31700028F7D123
:10B1400003A8801B20300190780701D5009801E00A
:10B15000012000900199884201DD401A00E00020A2
:10B160000027009006E002A8109AC05D0F99904752
:10B170006D1C7F1C0B988742F5DB04E0109A302091
:10B180000F9990476D1C0099481E00900029F5DC2E
:10B1900005E03078109A761C0F9990476D1C019944
:10B1A000481E01900029F4DC641C65E709280100B1
:10B1B000F8B54A002B4B520DD6182B4A0C460546C3
:10B1C000142E2BDA002E12DA284BFAF7B3F80022ED
:10B1D0001346FAF7DFFA40D2002C03DA0124E40721
:10B1E00000253AE02046284337D0214C14E0214F77
:10B1F0000B46F7403B402B4331D01C4BFAF79AF8F3
:10B2000000221346FAF7C6FA27D2002C03DD0120EC
:10B210000005F0400419BC4300251EE0332E1EDC5F
:10B2200033460027143BFF43DF40384217D00F4B13
:10B23000FAF72AF900221346FAF7ACFA0DD2002CDD
:10B240000ADD142E0CD03420811B012088404019C7
:10B25000A84200D2641C0546BD4321462846F8BDDD
:10B26000641CF9E701FCFFFF9C7500883CE4377E15
:10B270000000F03FFFFF0F0070B504467D20C000C6
:10B2800060430546284600F001F870BD002100BF6C
:10B2900040E000BF00BF00BF00BF00BF00BF00BF55
:10B2A00000BF00BF00BF00BF00BF00BF00BF00BFA6
:10B2B00000BF00BF00BF00BF00BF00BF00BF00BF96
:10B2C00000BF00BF00BF00BF00BF00BF00BF00BF86
:10B2D00000BF00BF00BF00BF00BF00BF00BF00BF76
:10B2E00000BF00BF00BF00BF00BF00BF00BF00BF66
:10B2F00000BF00BF00BF00BF00BF00BF00BF00BF56
:10B3000000BF00BF00BF00BF00BF00BF00BF00BF45
:10B3100000BF491C8142BCD370470000F0B585B026
:10B3200004460020049003902578607940008A4903
:10B33000085A02906078401E8849C6B20863042DFE
:10B3400001D0072D01D1012000E0002001902078DC
:10B3500082490873E07900280AD1084680690121F2
:10B36000890508437D4988610298C010029006E073
:10B370007A48806901218905884378498861207A63
:10B380007649487308468069217A09040322120429
:10B3900011400843714988610846002182690420F0
:10B3A00000F0B5FB6E492E20029A00F09FFB30465C
:10B3B000FFF788FD6B48405D810040186A494318DB
:10B3C000052207212B2000F0B7FB684901980B18D4
:10B3D00001220B21282000F0AFFB6248405D800075
:10B3E00063490A580C21282000F091FBE079800085
:10B3F00060494018A1794900425A0221272000F0F3
:10B4000075FB70005C490A5A0421272000F06EFB8E
:10B41000E079002805D164220621272000F066FB90
:10B420001EE0A07804280DD11020009010220621E3
:10B43000272000F05BFB6B4601222621272000F02D
:10B440007BFB0DE02820009020220621272000F021
:10B450004DFB6B4601222621272000F06DFB00BF2B
:10B46000300146494018E1788900425808212720D8
:10B4700000F04DFBA17A627A08021043002803D144
:10B480003F496172090AA172A17A637A08021843DE
:10B4900002462021272000F029FB3A480C210268AF
:10B4A000232000F034FB71003648001D425A04216D
:10B4B000232000F01BFBA07900280BD0E079324953
:10B4C000431801220021212000F036FB03200490C4
:10B4D000012003902807000F2901F02211400843A2
:10B4E00061788904032292041140084304990905F4
:10B4F000920011400843039949040122520411406B
:10B500000843217989051F2292051140084361797A
:10B51000C906C90EC906084307463A4600211F203E
:10B5200000F0F5FAA0786178084300040B4908613F
:10B5300008460069E17949030122D2031143084317
:10B5400006490861084600210269082000F0DFFA78
:10B55000002005B0F0BD00001CC0000890010020D4
:10B5600004280000C4BF00080200002020000020C2
:10B57000CCBF0008ECBF0008F8BF0008FCBF000803
:10B5800041100000E4BF00082200002038B5044646
:10B590000D460848808B0443224600212C2000F0F1
:10B5A000A5FA00956B46012206212C2000F0C4FA72
:10B5B00038BD00009001002010B5FFF771FC10BDF0
:10B5C00070B505460421362000F022F90446002D0E
:10B5D00003D00120C002044304E00121C902204637
:10B5E0008843044622460421362000F090FA70BDBC
:10B5F00038B54020009000210E2000F009F90446E3
:10B60000002211460E2000F082FA6B460122002132
:10B610000D2000F091FA084A00210F2000F077FA7F
:10B6200000F048FA224600210E2000F070FA0021B6
:10B630000248017338BD0000F8FF2724B001002044
:10B64000F0B585B006460420029000270020019046
:10B650005F494875086300215D48203041710173DE
:10B6600000205B4988834863886300F0EBF8584901
:10B67000086003E000F0E6F85549086054480068A7
:10B6800054498842F6D10020FFF73CFC524800782C
:10B69000242804DD504800780446243C0DE00621AF
:10B6A0004D480078F9F73AFD0621081A45014A4845
:10B6B0000078F9F733FD2C460C432006210408439B
:10B6C000210208432043039000211E20039A00F02A
:10B6D0001EFA02AB01220021242000F02DFA1E20C8
:10B6E000FFF798FC87B23812394988730420FFF7B6
:10B6F00091FC01900198C0B200280FD00220009068
:10B700006B46012212212D2000F016FA3048808B62
:10B710000121090308432E49888300BF00F092F8F5
:10B720002B4908600620FFF775FC2949486007206F
:10B73000FFF770FC26498860F806C00E08750846B9
:10B74000007D002801D1102008752149087D00F0F6
:10B750004BFAF007C00F002809D0FFF742FC1C4845
:10B76000808B0121C9020843194988830CE0052117
:10B77000362000F035F80546184805402A460521D0
:10B78000362000F0B3F900BF0120FFF7BBFB00211A
:10B79000042000F03DF80E4988610021262000F0C9
:10B7A00037F80546052080030543800005432A46F7
:10B7B0000021262000F0ABF900222621362000F0DF
:10B7C00095F900F03FF802490860002005B0F0BD8F
:10B7D000900100203001CADE01000020FFFD0000C2
:10B7E000F8B504460D46094FA9B2A0B26B46022235
:10B7F00000F02EF80646002E06D168464078010279
:10B8000068460078081887B23846F8BDFFFF000088
:10B81000FEB505460E460027FF43B1B2A8B201AB04
:10B82000042200F015F800900098002808D10324A5
:10B8300004E0380201A9095D4718641E002CF8DAFB
:10B840003846FEBD10B500210846FFF7E1FF10BDE8
:10B85000FFB581B006460C4617460025002C04D1E2
:10B8600029466D1C684646541AE040203043C2B257
:10B8700029466D1C684642547F2C04DC28466D1C0A
:10B8800069460C540CE0E0B28021084329466D1C47
:10B890006A4650546004020E28466D1C69460A54DC
:10B8A000A8B23A466946049B00F00CFB05B0F0BD17
:10B8B00070B504460D46164623462A4631461120E9
:10B8C000FFF7C6FF70BD10B50446234605220021D0
:10B8D0001520FFF7BDFF10BD10B501210620FFF7B1
:10B8E00097FF10BD10B504462346052200211720FE
:10B8F000FFF7AEFF10BD38B504460020009000F001
:10B90000D9F8FF250135002C01D0680005432A46EF
:10B9100000210D2000F0EAF8002C17D06B46012220
:10B9200003210F20FFF794FF6846007808210840A4
:10B9300000280BD0FFF75CFEFF2501352A460021C9
:10B940000D2000F0D3F80020C04338BD0020FCE7F4
:10B9500010B50446224601210A2000F0D8F810BD97
:10B9600070B5054600211A20FFF752FF0446240D4A
:10B9700024052803000B0443224600211A2000F06E
:10B98000C6F870BD10B50446224602492E2000F0CC
:10B99000ADF810BD0418000038B504466B4601220E
:10B9A00003210420FFF754FF002C16DD224600215E
:10B9B0000C2000F09BF8694608781021084300909D
:10B9C0000F488069090608430D4988616B460122CA
:10B9D0000321042000F0B0F810E069460878102137
:10B9E00088430090064880690906884304498861B5
:10B9F0006B4601220321042000F09EF838BD0000B0
:10BA00009001002010B5044622460021182000F0C5
:10BA10006DF810BDF8B50446002500200090002602
:10BA20000220204000280AD0802000906B4601228E
:10BA300000210D2000F080F801211D480173E0076E
:10BA4000C00F002826D069460878062108430090D8
:10BA50006B46012200210D2000F06EF803210F201B
:10BA6000FFF7BEFE06468120C0003040002801D10D
:10BA700000251AE0402000906B46012200210D2095
:10BA800000F05AF80020FFF79BFD002108480173E1
:10BA90004D1E0AE0694608780221084300906B4673
:10BAA000012200210D2000F047F82846F8BD0000D3
:10BAB000B00100201CB501AB012203210F20FFF7CC
:10BAC000C7FE694608798021084069460979402205
:10BAD00011404900884208D0012000906B460122A5
:10BAE00003210D2000F028F800BF1CBDF8B5054665
:10BAF0000E4614466846047021124170B1B2A8B2D5
:10BB00006B46022200F018F807463846F8BDFEB52D
:10BB100006460F461446002503E069464C55240AA4
:10BB20006D1C042DF9DBB9B2B0B26B46042200F0F3
:10BB300003F801900198FEBDFFB581B006460C46A2
:10BB400017460025002C07D180203043C2B2294679
:10BB50006D1C6846425419E0C0203043C2B22846EA
:10BB60006D1C69460A547F2C03DC28466D1C0C545E
:10BB70000CE0E0B28021084329466D1C6A4650540F
:10BB80006004020E28466D1C69460A54A8B23A4663
:10BB90006946049B00F0E4F905B0F0BD70B50446B9
:10BBA0000E461546281901218902884202DD00202F
:10BBB000C04370BDA21E334629460920FFF7BCFFD3
:10BBC0000020F6E770B504460D460648006920439C
:10BBD000A90508430646324600210820FFF797FFD3
:10BBE000002070BD9001002038B504466B4601224C
:10BBF0000E212B20FFF72CFE6846007841094901F1
:10BC00000091E106C90E68460078014300916B4639
:10BC100001220E212B20FFF78FFF38BD70B50146A2
:10BC2000002006E00A541E06140A34431B0A22466A
:10BC3000401C0428F6DB70BD13B50C4601231A46E0
:10BC400069460248FCF796FC00981CBD14170020BA
:10BC50007CB500210C460D466846FFF734FE0426ED
:10BC600008E0220E28021043240205466846805D43
:10BC70000443761E002EF4DA204629467CBD7CB5AE
:10BC800000210C460D466846FFF72CFE042608E00E
:10BC9000220E28021043240205466846805D0443B4
:10BCA000761E002EF4DA204629467CBDFBF734F9D7
:10BCB000FEF726FAFDF78EF8FDF76CF9FDF770F840
:10BCC000FDF7AEF9FDF782F9FDF722F80122D10365
:10BCD00005200007FBF70BF9FEF76AF8FCF7E0FE1A
:10BCE000F9F786FFF9F748FF0721FF204130FFF7FA
:10BCF0004DFC2E4800880A2148432D490880012226
:10BD0000110305200007FBF7F2F8C82229492A4849
:10BD1000FCF7BAFB002801D0F9F7AEFF45E0274851
:10BD2000007800283FD0FEF7EBF900202349087087
:10BD3000FAF716FA22490870084600780F280DDD38
:10BD4000012211031F48FBF7D2F8FEF76BFA00221D
:10BD5000012109031B48FBF7CAF80CE0012251033B
:10BD60001848FBF7C4F8FEF75DFA002201214903E9
:10BD70001448FBF7BCF8FCF791FD0D48008800283B
:10BD800004DD0B480088401E094908800E480078F1
:10BD900000280AD106480088002806D1012108465B
:10BDA000FBF750FB01E0FCF779FDB8E760010020EC
:10BDB00074010020F40C0020141700205101002011
:10BDC00050010020000400504500002000B585B05F
:10BDD0001748FBF770F914216846F9F7FCF9154884
:10BDE0000090032001900020029069460520000782
:10BDF000FAF77AFF69461048FAF776FF69460F4866
:10BE0000FAF772FF01210846FBF71CFBFF20013007
:10BE1000FBF7EAFA0A480068042108430849086069
:10BE20008815FBF7F3FAFBF7F9FA05B000BD00003F
:10BE30008C160020FFFF0000000400500008005096
:10BE40000070004010B5012292021B491B48F9F70F
:10BE50004AFF194800881A4988422CD008461649DA
:10BE6000088004208880FF20F530C8800A200881DF
:10BE7000002048811E20C04388810120C881002005
:10BE80000884088248828882C88208838883432085
:10BE9000C886022008877820488701208887C887BD
:10BEA00000210548403001844184818400200249FA
:10BEB000C88300F03BF810BDBC0D002000FC00085A
:10BEC000AA55000070B504460D4600211020052635
:10BED0003607B06200BF0DE0685C134EF06000BF33
:10BEE00011488068C007C00F0028F9D00E48C0680C
:10BEF0001870491CA142EFDB00210DE000200A4E22
:10BF0000F06000BF08488068C007C00F0028F9D063
:10BF10000548C0685854491C9142EFD310200526AB
:10BF20003607B061002070BD0030014010B500241C
:10BF300072B6012189020848F9F7BAFE0446002CBE
:10BF400006D00122920205490348F9F7A3FF0446EF
:10BF500062B6204610BD000000FC0008BC0D0020A9
:10BF600070B504460D460021102005263607B06244
:10BF700000BF0CE0685C124EF06000BF10488068A3
:10BF8000C007C00F0028F9D00D48C068491CA14265
:10BF9000F0DB00210CE0585C094EF06000BF08485F
:10BFA0008068C007C00F0028F9D00548C068491C48
:10BFB0009142F0D3102005263607B061002070BDF5
:10BFC000003001400000010203040005405C000055
:10BFD000A05C0400C06C0800805C0400E03F1E0010
:10BFE000E07D1E0007A9022570889B880A001600C4
:10BFF000010006000100020087008D002D001A31AB
:10C0000052001A339A001A351D011A376B003B3162
:10C01000BE003B335E013B3596023B370000995929
:10C020009959EB518F421E45142E0080EB51F52893
:10C030003333E13A703DE13AC235852BC2353333B3
:10C04000C235C235AE47E13A5138A330513800000D
:10C0500000000000000001020304060708090000B8
:10C06000000001020304030406080C10182030002D
:10C0700090C000080000002090010000E85900086E
:10C08000CCC0000890010020B01A000092AE000859
:10C0900021130704380D091E080540082609104021
:10C0A00008560A131D043B08BE0596D8BC4010086C
:10C0B0000430C8420114020214130909120202C911
:0CC0C00081A38C0A0249015220000000FC
:04000005080050C1DE
:00000001FF
